:100000000C9481040C949C040C949C040C949C040B
:100010000C949C040C949C040C949C040C949C04E0
:100020000C949C040C949C040C949C040C949C04D0
:100030000C94C1050C949C040C949C040C949C049A
:100040000C949C040C949C040C94DC090C943710C4
:100050000C9430070C949C040C949C040C949C0409
:100060000C949C040C949C040C949C040C949C0490
:100070000C949C040C949C040C949C04083B3BD76B
:100080004ABC846E023D2FC1FEBD9A31743DDA3DFB
:1000900083BE117FC73E4CBBE5BEAAAA6C3F800061
:1000A0000000555000000555000A9550000005520B
:1000B000000AA5500000054A000AA9500000052AC0
:1000C000000AAA50000004AA000AAA90000004AA8C
:1000D000000AAAA0000002AA000AAAA800000AAA10
:1000E000000A6AA800000AAD000A5AA800000AB572
:1000F000000A56A800000AD5000A55A800000B55B2
:10010000000A556800000D55000A555000000555BD
:10011000000AE00000000001000A5A00000000058B
:10012000000A54A000000015000A550A00000055FE
:10013000000A5540A0000155000A55500A00055517
:10014000000A555400A01555000A5555000A55558A
:10015000000A55554001F555000A555550055F55A3
:10016000000A5555541555F5000A55555555555F16
:10017000000A400000000000000310000000000022
:100180000003040000000000000301000000000064
:100190000003004000000000000300100000000009
:1001A0000003000400000000000300010000000044
:1001B00000030000400000000003000010000000E9
:1001C0000003000004000000000300000100000024
:1001D00000030000004000000003000000100000C9
:1001E00000030000000800000003000000020000FF
:1001F0000003000000008000000300000000200059
:1002000000030000000008000003000000000200DE
:100210000003000000000080000300000000002038
:1002200000030000000000080003000000000002BE
:100230000003000000000000800300000000000038
:100240002003000000000000080300000000000080
:100250000403400000000000000310000000000044
:100260000003040000000000000301000000000083
:100270000003004000000000000300100000000028
:100280000003000400000000000300010000000063
:100290000003000040000000000300001000000008
:1002A0000003000004000000000300000100000043
:1002B00000030000004000000003000000100000E8
:1002C000000300000008000000030000000200001E
:1002D0000003000000008000000300000000200078
:1002E00000030000000008000003000000000200FE
:1002F0000003000000000080000300000000002058
:1003000000030000000000080003000000000002DD
:100310000003000000000000800300000000000057
:10032000200300000000000008030000000000009F
:100330000403000000000000010340000000000072
:100340000003100000000000000304000000000093
:100350000003010000000000000300400000000056
:100360000003001000000000000300040000000073
:100370000003000100000000000300004000000036
:100380000003000010000000000300000400000053
:100390000003000001000000000300000040000016
:1003A000000300000010000000030000000800002F
:1003B00000030000000200000003000000008000B5
:1003C00000030000000020000003000000000800FF
:1003D0000003000000000200000300000000008095
:1003E00000030000000000200003000000000008DF
:1003F00000030000000000020003000000000000F5
:100400008003000000000000200300000000000046
:1004100008030000000000000403000000000000CA
:100420000103400000000000000310000000000075
:1004300000030400000000000003010000000000B1
:100440000003004000000000000300100000000056
:100450000003000400000000000300010000000091
:100460000003000040000000000300001000000036
:100470000003000004000000000300000100000071
:100480000003000000400000000300000010000016
:10049000000300000008000000030000000200004C
:1004A00000030000000080000003000000002000A6
:1004B000000300000000080000030000000002002C
:1004C0000003000000000080000300000000002086
:1004D000000300000000000800030000000000020C
:1004E0000003000000000000800300000000000086
:1004F00020030000000000000803000000000000CE
:100500000403400000000000000350000000000051
:10051000000354000000000000035500000000002C
:10052000000355400000000000035550000000008B
:100530000003555400000000000355550000000062
:1005400000035555400000000003555550000000C1
:100550000003555554000000000355555500000098
:1005600000035555554000000003555555500000F7
:1005700000035555555400000003555555550000CE
:10058000000355555555400000035555555550002D
:100590000003555555555400000355555555550004
:1005A0000003555555555540000355555555555063
:1005B000000355555555555400035555555555553A
:1005C00000035555555555554003555555555555E9
:1005D0005003555555555555540355555555555575
:1005E0005503555555555555540355555555555560
:1005F0005003555555555555400355555555555569
:1006000000035555555555540003555555555550EE
:100610000003555555555540000355555555550042
:100620000003555555555400000355555555500078
:1006300000035555555540000003555555550000CC
:100640000003555555540000000355555550000002
:100650000003555555400000000355555500000056
:10066000000355555400000000035555500000008C
:1006700000035555400000000003555500000000E0
:100680000003555400000000000355500000000016
:10069000000355400000000000035500000000006A
:1006A00000035400000000000003500000000000A0
:1006B00000034000000000000003000000000000F4
:1006C00000038000000000000203A0000000000002
:1006D0000A03A800000000002A03AA00000000008E
:1006E000AA03AA8000000002AA03AAA00000000A30
:1006F000AA03AAA80000002AAA03AAAA000000AA26
:10070000AA03AAAA800002AAAA03AAAAA0000AAA67
:10071000AA03AAAAA8002AAAAA03AAAAAA00AAAA5D
:10072000AA03AAAAAA82AAAAAA03AAAAAAAAAAAA9F
:10073000AA03AAAAAA82AAAAAA03AAAAAA00AAAA39
:10074000AA03AAAAA8002AAAAA03AAAAA0000AAAD7
:10075000AA03AAAA800002AAAA03AAAA000000AAC1
:10076000AA03AAA80000002AAA03AAA00000000A5F
:10077000AA03AA8000000002AA03AA000000000049
:10078000AA03A800000000002A03A0000000000047
:100790000A038000000000000203000000000000C7
:1007A00000038000000000000203200000000000A1
:1007B0000803080000000000200302000000000001
:1007C00080030080000000020003002000000008F9
:1007D0000003000800000020000300020000008069
:1007E0000003000080000200000300002000080059
:1007F0000003000008002000000300000200800049
:100800000003000000820000000300000028000038
:10081000000300000000000000035400000000007E
:10082000000A015000000000000A0005400000001E
:10083000000A000015000000000A0000005400003B
:10084000000A000000015000000A000000000540FE
:10085000000A000000000015000A00000000000A65
:10086000000A0000000000A8000A000000000A8042
:10087000000A00000002A000000A000000A800001A
:10088000000A00002A000000000A000A80000000A0
:10089000000A02A000000000000AA80000000000FA
:1008A000000AC00000000003000A3C000000000035
:1008B000000A03C000000000000A003C0000000025
:1008C000000A0003C0000000000A00003C00000015
:1008D000000A000003C00000000A0000003C000005
:1008E000000A00000003C000000A000000003C00F5
:1008F000000A0000000003C0000A00000000003CE5
:10090000000A11241FBECFEFD0E1DEBFCDBF11E042
:10091000A0E0B1E0ECE1F1E302C005900D92AC384B
:10092000B107D9F712E0ACE8B1E001C01D92A83DD3
:10093000B107E1F70C94B9040C940000CF93DF9356
:10094000CDB7DEB7E4E2F0E086E08083EAE2F0E0F3
:1009500088E88083EBE2F0E080E38083E7E2F0E088
:100960008CEF8083E1E2F0E08FEF8083DF91CF9125
:100970000895CF93DF93CDB7DEB722970FB6F894E3
:10098000DEBF0FBECDBF0E949E040E94B2050E9432
:100990006C060E94C70980EF9DE09093BD01809393
:1009A000BC018CEA9CE09093BF018093BE0182E67B
:1009B0009DE09093C1018093C00181E59CE09093FC
:1009C000C3018093C2018BE69EE09093C5018093A2
:1009D000C40189ED9EE09093C7018093C60189ED23
:1009E0009EE09093C9018093C8011A82198211C0B8
:1009F00029813A8189819A81FC01E25FFE4F8081E1
:100A0000F901E759FD4F808389819A8101969A8384
:100A1000898389819A818730910554F37894ABE278
:100A2000B0E0EBE2F0E0808188608C9380919801E7
:100A30008823E1F310929801ABE2B0E0EBE2F0E042
:100A4000808180688C93F8941A82198211C0298160
:100A50003A8189819A81FC01E050FF4F8081F90140
:100A6000E759FD4F808389819A8101969A83898312
:100A700089819A818730910554F378948091980107
:100A80008823E1F3109298011A82198211C02981FA
:100A90003A8189819A81FC01E95FFE4F8081F901E9
:100AA000E759FD4F808389819A8101969A838983D2
:100AB00089819A818730910554F380919801882328
:100AC000E1F310929801ABE2B0E0EBE2F0E080815C
:100AD000877F8C938CE191E00E94DC0700C08091BD
:100AE0009C01813011F40E9419118091950181308F
:100AF00001F580917A01882369F480919B019927FF
:100B0000880F991FFC01E454FE4F0190F081E02D05
:100B100009950DC08091930190919401880F991FC0
:100B2000FC01E454FE4F0190F081E02D09951092F4
:100B3000950180919601813031F40E947C0F1092D2
:100B400096010E94721080919801813041F60E94B6
:100B5000B00880919A01813011F40E94CE0B10925E
:100B60009801BDCFCF93DF93CDB7DEB7E1E8F0E0DA
:100B700082E48083EFE6F0E080E28083DF91CF9132
:100B800008951F920F920FB60F9211242F933F9347
:100B90004F935F936F937F938F939F93AF93BF9385
:100BA000EF93FF93CF93DF93CDB7DEB780919E0194
:100BB00090919F010097B1F4E6E8F0E08081918187
:100BC0009093A5018093A401A1E8B0E0E1E8F0E0F2
:100BD00080818F7B8C9381E090E090939F01809344
:100BE0009E0167C0E6E8F0E0808191819093A301C7
:100BF0008093A201A1E8B0E0E1E8F0E080818064A8
:100C00008C932091A2013091A3018091A401909135
:100C1000A501A901481B590BCA019093A10180931A
:100C2000A00110929F0110929E018091A0019091CD
:100C3000A101845C99409093A1018093A0018091CF
:100C4000A0019091A10120E931E0B9010E94F916BB
:100C5000CB019093A1018093A0018091A00190917C
:100C6000A101992324F41092A1011092A001809176
:100C7000A0019091A1018730910534F086E090E0C9
:100C80009093A1018093A0012091A0013091A10136
:100C900080919301909194012817390751F0109297
:100CA000AF018091A0019091A10190939401809354
:100CB0009301DF91CF91FF91EF91BF91AF919F9100
:100CC0008F917F916F915F914F913F912F910F90F5
:100CD0000FBE0F901F901895CF93DF93CDB7DEB75F
:100CE000E0ECF0E01082E1ECF0E088E98083E2ECF7
:100CF000F0E086E08083E4ECF0E085E18083E5ECE1
:100D0000F0E01082DF91CF910895CF93DF93CDB7BC
:100D1000DEB764970FB6F894DEBF0FBECDBF83E297
:100D20008F83188683E689871A861B8685E090E084
:100D30009E838D831C821B821A82198215C0298191
:100D40003A81CE010796FC01E20FF31F8081282F24
:100D500033278B819C81820F931F9C838B83898196
:100D60009A8101969A83898329813A818D819E8116
:100D70002817390724F38B819C8120E030E1B901E9
:100D80000E940D179C838B838D819E819A8B898B0A
:100D90008B819C819C8B8B8B8B899C8999232CF4D8
:100DA0008B899C89CF969C8B8B8B8B899C89082EF9
:100DB000892F000C881F990B000C881F991F282F62
:100DC000235CCE010796E989FA89E80FF91F208391
:100DD0008D819E8101969E838D83ED81FE818B8125
:100DE0009C8120E430E0B9010E940D17282F235C7C
:100DF000CE010796E80FF91F20838D819E81019611
:100E00009E838D832D813E81CE010796FC01E20FEA
:100E1000F31F8DE080838D819E8101969E838D835B
:100E20001A8219820FC029813A81CE010796FC01EE
:100E3000E20FF31F80810E94BC0789819A8101968D
:100E40009A83898389819A818830910564F36496B5
:100E50000FB6F894DEBF0FBECDBFDF91CF910895DE
:100E60001F920F920FB60F9211242F933F938F93DF
:100E70009F93AF93BF93EF93FF93CF93DF93CDB740
:100E8000DEB72397DEBFCDBFE6ECF0E0808189833B
:100E900089818D30C9F48091A6018130A9F4ABE23B
:100EA000B0E0EBE2F0E08081877F8C931092A601A6
:100EB00081E080939C01809166029927FC01E253B6
:100EC000FE4F8981808345C08091A601282F33275A
:100ED0003B832A838A819B81009731F02A813B8161
:100EE0002130310511F135C08981833271F480914F
:100EF0009C01882351F481E08093A601ABE2B0E02D
:100F0000EBE2F0E0808188608C9310926602209181
:100F10006602822F9927FC01E253FE4F898180836C
:100F2000822F8F5F8093660214C08091660299279A
:100F3000FC01E253FE4F89818083809166028639ED
:100F400030F4809166028F5F8093660202C0109237
:100F5000A6012396F894DEBFCDBFDF91CF91FF911C
:100F6000EF91BF91AF919F918F913F912F910F90F2
:100F70000FBE0F901F901895CF93DF93CDB7DEB7BC
:100F800021970FB6F894DEBF0FBECDBF8983E0EC8A
:100F9000F0E080819927807290700097C1F3E6ECB1
:100FA000F0E08981808321960FB6F894DEBF0FBEF2
:100FB000CDBFDF91CF910895CF93DF93CDB7DEB74B
:100FC00026970FB6F894DEBF0FBECDBF9E838D83EC
:100FD0008D819E81DC01FD0101900020E9F73197B0
:100FE000CF018A1B9B0B9C838B831A8219820FC0B3
:100FF00029813A818D819E81F901E80FF91F808155
:101000000E94BC0789819A8101969A8389832981EC
:101010003A818B819C818217930750F78091370129
:101020000E94BC07809138010E94BC0726960FB62B
:10103000F894DEBF0FBECDBFDF91CF910895CF935F
:10104000DF93CDB7DEB766970FB6F894DEBF0FBE5D
:10105000CDBF9E8B8D8B8D899E894AE050E09E018D
:101060002F5F3F4FB9010E94C816CE0101960E9422
:10107000DC0766960FB6F894DEBF0FBECDBFDF91DA
:10108000CF910895CF93DF93CDB7DEB76E970FB6AC
:10109000F894DEBF0FBECDBF80E489838DE68A83DE
:1010A0001B8280917A01813079F482E78B832091D1
:1010B000930130919401CE010B964AE050E0BC01BF
:1010C000C9010E94C8160EC088E68B8380919B01DF
:1010D000282F3327CE010B964AE050E0BC01C9010E
:1010E0000E94C8161C82CE010B96DC01FD01019006
:1010F0000020E9F73197CF018A1B9B0B9E01255FEA
:101100003F4FAC01B901CE0101960E94B816CE0145
:101110000196DC01FD0101900020E9F731979F0164
:101120002A1B3B0BCE010196820F931FFC0183E229
:1011300090E091838083CE0101960E94DC0780912C
:1011400037010E94BC07809138010E94BC076E964F
:101150000FB6F894DEBF0FBECDBFDF91CF910895DB
:10116000CF93DF93CDB7DEB76E970FB6F894DEBF9F
:101170000FBECDBF2091980230919902CE010B96FF
:101180004AE050E0BC01C9010E94C81680E489838E
:101190008EE48A8380E38B831C82CE010B96DC0174
:1011A000FD0101900020E9F73197CF018A1B9B0BCD
:1011B0009E01255F3F4FAC01B901CE0101960E940F
:1011C000B816CE010196DC01FD0101900020E9F77F
:1011D00031979F012A1B3B0BCE010196820F931F73
:1011E000FC0183E290E091838083CE0101960E940E
:1011F000DC0720919A0230919B02CE010B964AE0C7
:1012000050E0BC01C9010E94C81680E4898382E5D0
:101210008A8381E38B831C82CE010B96DC01FD0166
:1012200001900020E9F73197CF018A1B9B0B9E01AB
:10123000255F3F4FAC01B901CE0101960E94B8165F
:10124000CE010196DC01FD0101900020E9F7319704
:101250009F012A1B3B0BCE010196820F931FFC01BD
:1012600083E290E091838083CE0101960E94DC07A7
:101270002091870230918802CE010B964AE050E01F
:10128000BC01C9010E94C81680E4898386E48A8370
:1012900082E38B831C82CE010B96DC01FD01019061
:1012A0000020E9F73197CF018A1B9B0B9E01255F38
:1012B0003F4FAC01B901CE0101960E94B816CE0194
:1012C0000196DC01FD0101900020E9F731979F01B3
:1012D0002A1B3B0BCE010196820F931FFC0183E278
:1012E00090E091838083CE0101960E94DC072091DB
:1012F0008C0230918D02CE010B964AE050E0BC0189
:10130000C9010E94C81680E4898387E78A8381E344
:101310008B831C82CE010B96DC01FD010190002025
:10132000E9F73197CF018A1B9B0B9E01255F3F4F49
:10133000AC01B901CE0101960E94B816CE0101960A
:10134000DC01FD0101900020E9F731979F012A1B84
:101350003B0BCE010196820F931FFC0183E290E0CC
:1013600091838083CE0101960E94DC078091370132
:101370000E94BC07809138010E94BC076E960FB690
:10138000F894DEBF0FBECDBFDF91CF910895CF930C
:10139000DF93CDB7DEB7A5E4B0E0E5E4F0E080810F
:1013A00082608C93AEE6B0E0EEE6F0E08081816092
:1013B0008C93DF91CF9108951F920F920FB60F92E9
:1013C00011242F933F938F939F93AF93BF93EF93EA
:1013D000FF93CF93DF93CDB7DEB72297DEBFCDBFAC
:1013E0008091A9019091AA0101969093AA018093FE
:1013F000A9018091A9019091AA018436910519F55E
:1014000081E0809395011092AA011092A901809128
:1014100070028F5F8093700280917002843629F48D
:101420001092700281E080939801809168028F5F32
:1014300080936802809168028A3029F410926802D1
:1014400081E0809396018091A701282F33273A836A
:10145000298389819A818530910509F4D2C0298137
:101460003A812630310524F589819A8182309105AF
:1014700009F47DC029813A812330310564F48981E2
:101480009A81009709F43FC029813A8121303105C2
:1014900009F451C067C189819A818330910509F4AB
:1014A0007DC029813A812430310509F493C05AC1A5
:1014B00089819A818830910509F4F2C029813A81A5
:1014C000293031056CF489819A818630910509F4BF
:1014D000B4C029813A812730310509F4C5C042C121
:1014E00089819A818A30910509F40DC129813A8157
:1014F0002A3031050CF4EBC089819A818B3091053B
:1015000009F417C12FC18091A8018F5F8093A801B2
:101510008091A801883008F425C11092A801A8E2A2
:10152000B0E0E8E2F0E090818FE789238C9381E0DE
:101530008093A70117C18091A8018F5F8093A801B4
:101540008091A801883008F40DC11092A801E2E250
:10155000F0E0809169028083A8E2B0E0E8E2F0E088
:10156000808184608C9382E08093A701FBC080918E
:10157000A8018F5F8093A8018091A801883008F4AA
:10158000F1C01092A801A8E2B0E0E8E2F0E08081AA
:101590008B7F8C9383E08093A701E4C08091A801A6
:1015A0008F5F8093A8018091A801883008F4DAC089
:1015B0001092A801E2E2F0E080916A028083A8E242
:1015C000B0E0E8E2F0E0808188608C9384E0809372
:1015D000A701C8C08091A8018F5F8093A801809166
:1015E000A801883008F4BEC01092A801A8E2B0E0BB
:1015F000E8E2F0E08081877F8C9385E08093A7010B
:10160000B1C08091A8018F5F8093A8018091A8014B
:10161000883008F4A7C01092A801E2E2F0E08091BF
:101620006B028083A8E2B0E0E8E2F0E080818061B4
:101630008C9386E08093A70195C08091A8018F5F6D
:101640008093A8018091A801883008F48BC0109283
:10165000A801A8E2B0E0E8E2F0E080818F7E8C9300
:1016600087E08093A7017EC08091A8018F5F80935F
:10167000A8018091A801883008F474C01092A801D4
:10168000E2E2F0E080916C028083A8E2B0E0E8E260
:10169000F0E0808180628C9388E08093A70162C033
:1016A0008091A8018F5F8093A8018091A801883064
:1016B00008F458C01092A801A8E2B0E0E8E2F0E017
:1016C00080818F7D8C9389E08093A7014BC08091AE
:1016D000A8018F5F8093A8018091A801883008F449
:1016E00041C01092A801E2E2F0E080916D02808397
:1016F000A8E2B0E0E8E2F0E0808180648C938AE0C8
:101700008093A7012FC08091A8018F5F8093A801CB
:101710008091A801883030F11092A801A8E2B0E0D1
:10172000E8E2F0E080818F7B8C938BE08093A701CF
:1017300019C08091A8018F5F8093A8018091A801B2
:10174000883080F01092A801E2E2F0E080916E0211
:101750008083A8E2B0E0E8E2F0E0808180688C93CA
:101760001092A7012296F894DEBFCDBFDF91CF91F2
:10177000FF91EF91BF91AF919F918F913F912F91E9
:101780000F900FBE0F901F901895CF93DF93CDB79A
:10179000DEB780919901DF91CF910895CF93DF93C8
:1017A000CDB7DEB78091AE01813059F4ABE2B0E045
:1017B000EBE2F0E090818FE789238C931092AE01E9
:1017C0000AC0ABE2B0E0EBE2F0E0808180688C938D
:1017D00081E08093AE01DF91CF910895CF93DF93A5
:1017E000CDB7DEB722970FB6F894DEBF0FBECDBFE0
:1017F0008A8319828A81992781709070882319F0D1
:101800008981806889838A81992782709070009786
:1018100019F08981806489838A8199278470907006
:10182000009719F08981806289838A81992788705D
:101830009070009719F08981806189838A81992746
:1018400080719070009719F08981886089838A81FE
:10185000992780729070009719F08981846089833C
:101860008A81992780749070009719F0898182602D
:1018700089838A8188231CF4898181608983898195
:10188000992722960FB6F894DEBF0FBECDBFDF9129
:10189000CF910895CF93DF93CDB7DEB7DF91CF918E
:1018A00008950F931F93CF93DF93CDB7DEB72297A1
:1018B0000FB6F894DEBF0FBECDBF8091B201882372
:1018C00009F5F8941A82198213C009811A81898155
:1018D0009A81FC01E050FF4F80810E94EE0BF801DD
:1018E000E759FD4F808389819A8101969A83898384
:1018F00089819A818730910544F3789481E08093BF
:10190000B2011FC0F8941A82198213C009811A818A
:1019100089819A81FC01E95FFE4F80810E94EE0B74
:10192000F801E759FD4F808389819A8101969A8356
:10193000898389819A818730910544F37894109244
:10194000B20122960FB6F894DEBF0FBECDBFDF9175
:10195000CF911F910F9108950F931F93CF93DF9312
:10196000CDB7DEB726970FB6F894DEBF0FBECDBF5A
:10197000F8941D821C8229C080918E0290918F0262
:10198000880F991F880F991F880F991F9C018C81C0
:101990009D81280F391F82EA98E0820F931F9B8355
:1019A0008A83EA81FB818491898389818E830C817A
:1019B0001D818E810E94EE0BF801E759FD4F808357
:1019C0008C819D8101969D838C838C819D81873044
:1019D000910594F2789426960FB6F894DEBF0FBE68
:1019E000CDBFDF91CF911F910F9108950F931F935A
:1019F000CF93DF93CDB7DEB726970FB6F894DEBF4F
:101A00000FBECDBF80917A01813029F48091AF0162
:101A10008093B10104C08091B0018093B1011E8216
:101A20001D821FC08091B1019927880F991F880FCF
:101A3000991F880F991F9C018D819E81280F391F46
:101A400082EA90E0820F931F9B838A83EA81FB8165
:101A50008491898389818C838D819E8101969E8367
:101A60008D838D819E8187309105E4F20D811E81E9
:101A70008C810E94EE0BF801E759FD4F8083809125
:101A8000B1018F5F8093B1018091B1018E3010F070
:101A90001092B10180917A01813029F48091B101D5
:101AA0008093AF0104C08091B1018093B00126966C
:101AB0000FB6F894DEBF0FBECDBFDF91CF911F915F
:101AC0000F9108950F931F93CF93DF93CDB7DEB798
:101AD00029970FB6F894DEBF0FBECDBF80913901B4
:101AE00081508093390180913901882309F06DC0BC
:101AF00080917A01813029F48091AF018093B10106
:101B000004C08091B0018093B1018091B101992707
:101B1000880F991F880F991F880F991F9C0182E1D8
:101B200091E00796820F931F9E838D83ED81FE8146
:101B300084918C838C81809339011986188628C002
:101B40008091B1019927880F991F880F991F880FDD
:101B5000991F9C0188859985280F391F82E191E0A2
:101B6000820F931F9B838A83EA81FB8184918983FF
:101B700089818F83088519858F810E94EE0BF8017A
:101B8000E759FD4F808388859985019699878887D5
:101B900088859985873091059CF28091B1018F5F8E
:101BA0008093B1018091B1018C3010F01092B1019D
:101BB00080917A01813029F48091B1018093AF0145
:101BC00004C08091B1018093B00129960FB6F894BA
:101BD000DEBF0FBECDBFDF91CF911F910F91089552
:101BE0000F931F93CF93DF93CDB7DEB723970FB635
:101BF000F894DEBF0FBECDBF809139018150809334
:101C0000390180913901882309F05AC080917A0105
:101C1000813029F48091AF018093B10104C080919B
:101C2000B0018093B1018091B1019927880F991F6C
:101C3000880F991F880F991FFC01EF5BFE4F808171
:101C4000809339011B821A821EC00A811B818091F8
:101C5000B10199272A813B81880F991F880F991F0D
:101C6000880F991F820F931FFC01E65CFE4F808155
:101C70000E94EE0BF801E759FD4F80838A819B811A
:101C800001969B838A838A819B8187309105ECF240
:101C90008091B1018F5F8093B1018091B101883053
:101CA00011F41092B10180917A01813029F4809170
:101CB000B1018093AF0104C08091B1018093B00164
:101CC00023960FB6F894DEBF0FBECDBFDF91CF9144
:101CD0001F910F9108950F931F93CF93DF93CDB76B
:101CE000DEB726970FB6F894DEBF0FBECDBF80914A
:101CF0007A01813029F48091AF018093B10104C051
:101D00008091B0018093B101F8941E821D8228C099
:101D10008091AF019927880F991F880F991F880F0D
:101D2000991F9C018D819E81280F391F8AE198E0BF
:101D3000820F931F9B838A83EA81FB81849189832D
:101D400089818C830D811E818C810E94EE0BF801AC
:101D5000E759FD4F80838D819E8101969E838D83FF
:101D60008D819E81873091059CF278948091AF019E
:101D70008F5F8093AF018091AF01813110F010929D
:101D8000AF0180917A01813029F48091B101809373
:101D9000AF0104C08091B1018093B00126960FB6C7
:101DA000F894DEBF0FBECDBFDF91CF911F910F9191
:101DB00008950F931F93CF93DF93CDB7DEB7299785
:101DC0000FB6F894DEBF0FBECDBF809139018150B0
:101DD0008093390180913901882309F06DC0809189
:101DE0007A01813029F48091AF018093B10104C060
:101DF0008091B0018093B1018091AF019927880F44
:101E0000991F880F991F880F991F9C0182E791E005
:101E10000796820F931F9E838D83ED81FE818491AF
:101E20008C838C81809339011986188628C0809113
:101E3000AF019927880F991F880F991F880F991F45
:101E40009C0188859985280F391F82E791E0820FD0
:101E5000931F9B838A83EA81FB8184918983898193
:101E60008F83088519858F810E94EE0BF801E75951
:101E7000FD4F808388859985019699878887888515
:101E80009985863091059CF28091AF018F5F809398
:101E9000AF018091AF01873D10F01092AF018091AA
:101EA0007A01813029F48091B1018093AF0104C09F
:101EB0008091B1018093B00129960FB6F894DEBFEE
:101EC0000FBECDBFDF91CF911F910F910895CF939A
:101ED000DF93CDB7DEB70E9414128091CC019091B0
:101EE000CD018091CC019091CD018091CC01909158
:101EF000CD01DF91CF910895CF93DF93CDB7DEB7BA
:101F000022970FB6F894DEBF0FBECDBFE9E2F0E036
:101F100080819927807290700097B9F58091B30104
:101F20008F5F8093B301ABE2B0E0EBE2F0E0808141
:101F300088608C9381E08093B5018091B3018530F6
:101F400079F5ABE2B0E0EBE2F0E08081877F8C9343
:101F50001092B50180917A01813041F41092B00164
:101F600010927A0181E080939A011AC081E08093F7
:101F70007A011092AF0110929A01ABE2B0E0EBE26D
:101F8000F0E0808180688C930BC01092B301ABE2CB
:101F9000B0E0EBE2F0E08081877F8C931092B50196
:101FA000E9E2F0E08081992780719070009779F5DF
:101FB00080917A01882309F046C0ABE2B0E0EBE201
:101FC000F0E0808188608C9381E08093B6018091FD
:101FD000B4018F5F8093B4018091B401853099F58D
:101FE000ABE2B0E0EBE2F0E08081877F8C9310926F
:101FF000B60180919B018F5F80939B0180919B0133
:10200000873011F410929B011092B0011CC0109205
:10201000B4018091B5011A82882311F481E08A838A
:102020008091B6011982882311F491E099838A8105
:1020300099818923882339F0ABE2B0E0EBE2F0E04C
:102040008081877F8C9322960FB6F894DEBF0FBEF7
:10205000CDBFDF91CF910895CF93DF93CDB7DEB79A
:10206000ECE4F0E082EC8083DF91CF9108951F9241
:102070000F920FB60F9211242F933F938F939F933C
:10208000AF93BF93EF93FF93CF93DF93CDB7DEB7BB
:102090008091B70199279C0180917B0190917C01EF
:1020A000D901A80FB91FEEE4F0E080818C938091F4
:1020B000B7018F5F8093B7018091B701883019F421
:1020C00087E08093B701DF91CF91FF91EF91BF91AE
:1020D000AF919F918F913F912F910F900FBE0F90D5
:1020E0001F901895EF92FF920F931F93CF93DF935A
:1020F000CDB7DEB780919A0290919B029095819521
:102100009F4F9093950280939402809198029091B2
:102110009902AA2797FDA095BA2FBC01CD010E9474
:102120003E147B018C018091940290919502AA2724
:1021300097FDA095BA2FBC01CD010E943E14DC0191
:10214000CB01A8019701BC01CD010E945717DC010A
:10215000CB018093900290939102A0939202B0934E
:1021600093028091900290919102A0919202B0917D
:10217000930220E030E044E353E4BC01CD010E942F
:102180006612DC01CB017C018D0180917D01909173
:102190007E01A0917F01B09180019C01AD01C80139
:1021A000B7010E948413DC01CB01BC01CD010E9468
:1021B000A714DC01CB0190938D0280938C02809157
:1021C0008C0290918D02992354F480918C0290910D
:1021D0008D0288599E4F90938D0280938C0280913E
:1021E0008C0290918D022EE130E0B9010E940D1712
:1021F000CB0190938F0280938E0280918E029091FA
:102200008F02992324F410928F0210928E028091F3
:102210008E0290918F028C30910524F010928F02E3
:1022200010928E02DF91CF911F910F91FF90EF904E
:102230000895CF93DF93CDB7DEB764970FB6F894C8
:10224000DEBF0FBECDBF83E090E09C8B8B8B1A82EC
:10225000198283E990E09C838B8310929C0180918A
:10226000D001843409F0D7C0CFC08B899C89FC0190
:10227000E253FE4F80819927CD979A8B898B8B896A
:102280009C8901969C8B8B8B8B899C89FC01E253EA
:10229000FE4F80819927CD97988B8F878B899C895A
:1022A00001969C8B8B8B8B899C89FC01E253FE4FA2
:1022B00080819927CD979E878D878B899C890196F0
:1022C0009C8B8B8B8B899C89FC01E253FE4F808118
:1022D0009927CD979C878B878B899C8901969C8BAE
:1022E0008B8B89899A899C01220F331F220F331F00
:1022F0008F859889959587959595879595958795D7
:1023000095958795822B932B9A8789878F859889B6
:102310008F7090709C0122953295307F3227207FFC
:1023200032278D859E859595879595958795822BE6
:10233000932B98878F838D859E85837090709C01E9
:102340000024369527950794369527950794322FC4
:10235000202D8B859C85822B932B9E838D838B8157
:102360009C8101979C838B838B819C812FEF8F3F76
:10237000920709F44EC089819A819C018091810164
:1023800090918201F901E80FF91F89858083898185
:102390009A8101969A8389838B819C8101979C8382
:1023A0008B838B819C812FEF8F3F920791F18981E5
:1023B0009A819C018091810190918201F901E80F3D
:1023C000F91F8F81808389819A8101969A838983FD
:1023D0008B819C8101979C838B838B819C812FEFC8
:1023E0008F3F9207B1F089819A819C018091810190
:1023F00090918201F901E80FF91F8D818083898115
:102400009A8101969A8389838B819C81009709F038
:102410002CCF0E94141264960FB6F894DEBF0FBE44
:10242000CDBFDF91CF910895CF93DF93CDB7DEB7C6
:102430008091A2029091A30290936502809364021E
:1024400020916402309165028091CA019091CB0184
:10245000A901481B590BCA019093BB018093BA0193
:1024600080916402909165029093CB018093CA01A0
:102470002091B8013091B9018091BA019091BB01CE
:10248000820F931F9093B9018093B80180919D01B1
:102490008430A1F410929D018091B8019091B9010E
:1024A00025E030E0B9010E940D17CB019093CD01DA
:1024B0008093CC011092B9011092B80180919D01D6
:1024C0008F5F80939D01DF91CF910895A0E2B0E0EE
:1024D000ECE6F2E10C94201769837A838B839C836A
:1024E0002D833E834F8358878E01075E1F4FB801AF
:1024F000CE0101960E941916F1E1EF2EF12CEC0E9F
:10250000FD1EB701CE0105960E941916898D8230F5
:1025100078F09989923040F420E09A8D8A89981356
:1025200021E02A8BB701E9C0843051F4923061F088
:1025300020E09A8D8A89981321E02A8FB801DDC0A6
:10254000943029F4823041F763E871E0D6C08230DC
:1025500079F3923009F32D8D3E8D4F8D58A18D89E1
:102560009E89AF89B88D222433242101AA24BB245B
:102570006501EE24FF24870160E070E00DC06F5F0D
:102580007F4F6032710599F1880F991FAA1FBB1FF9
:10259000569547953795279520FF19C0280E391E67
:1025A0004A1E5B1E662477244301281639064A0614
:1025B0005B0628F4E1E06E2E712C812C912CAE0C80
:1025C000BF1CC01ED11EA60CB71CC81CD91CEE0C0B
:1025D000FF1C001F111FB7FFD2CFE1E06E2E712C40
:1025E000812C912CE628F72808291929C8CF8B8D32
:1025F0009C8D2B893C89820F931F02969C878B8729
:102600001A869A8D8A89981711F081E08A87D7FEF9
:1026100017C08B859C85A0FE0CC0569447943794B8
:10262000279420E030E040E050E8222A332A442A70
:10263000552AD694C794B794A79401969C878B8704
:1026400030E0A31630E0B30630E0C30630E4D30632
:1026500018F58B859C850EC0220C331C441C551C20
:10266000019720E0A21620E0B20620E0C20620E496
:10267000D20680F4AA0CBB1CCC1CDD1C57FEECCF90
:1026800031E0632E712C812C912CA628B728C82804
:10269000D928E2CF9C878B87D601C5018F779070B0
:1026A000A070B07080349105A105B10551F0AD86E0
:1026B000BE86CF86D88A83E08987BE01675F7F4F59
:1026C0001CC0A7FCF4CF211431044104510479F358
:1026D00080E490E0A0E0B0E0A80EB91ECA1EDB1EA8
:1026E00080E8682E8FEF782E8FEF882E8FEF982E50
:1026F000A620B720C820D920DACFCB010E94F7143A
:10270000E2E1A0960C943C17A8E1B0E0EAE8F3E11E
:102710000C94261769837A838B839C832D833E8355
:102720004F835887B1E18B2E912C8C0E9D1EB401E6
:10273000CE0101960E9419168E01075F1F4FB80146
:10274000CE0105960E9419162989223008F46AC024
:102750003985323008F468C08A899A8589278A8B3E
:10276000243009F463C0223009F460C0343041F4ED
:102770001D8A1E8A1F8A188E1C8A1B8AB40177C084
:10278000323009F458C06B897C898B859C85681B25
:10279000790B7C8B6B8B2D893E894F89588DED840D
:1027A000FE840F8518892E153F054007510740F418
:1027B000220F331F441F551F615070407C8B6B8B61
:1027C00080E090E0A0E0B0E4AA24BB24650160E0D2
:1027D00070E02E153F054007510740F0A82AB92A9E
:1027E000CA2ADB2A2E193F09400B510BB695A79533
:1027F00097958795220F331F441F551F6F5F7F4F9B
:102800006F31710531F7D601C5018F779070A070D7
:10281000B07080349105A105B10589F0AD8ABE8AFA
:10282000CF8AD88EB40123C0B80121C03217D1F7A6
:1028300063E871E01CC084E0898BB40118C0A7FC78
:10284000EDCF211531054105510541F380E490E0BC
:10285000A0E0B0E0A80EB91ECA1EDB1E80E89FEF04
:10286000AFEFBFEFA822B922CA22DB22D7CFCB011C
:102870000E94F714ECE068960C944217A8E0B0E0D0
:10288000E4E4F4E10C942F179B01AC0183E089830D
:102890001A8257FD51C0211531054105510539F402
:1028A00082E08983CE0101960E94F7144CC0EEE1CC
:1028B000F0E0FC83EB838A818823C9F1203010E0AB
:1028C000310710E0410710E85107C9F1882799271F
:1028D000DC01821B930BA40BB50B8D839E83AF830E
:1028E000B8872D813E814F815885203080E03807A0
:1028F00080E0480780E45807A8F6EB81FC81DA0104
:10290000C901880F991FAA1FBB1F31979C01AD01F8
:10291000803010E0910710E0A10710E4B10778F3D0
:10292000FC83EB838D839E83AF83B887BBCF2D83DE
:102930003E834F835887D5CF81E08A83ACCF60E058
:1029400070E080E09FECE3E028960C944B17ACE03D
:10295000B0E0EDEAF4E10C94301769837A838B835D
:102960009C83BE016B5F7F4FCE0101960E941916BA
:102970008D81823061F0823050F0843069F48E8134
:10298000882359F52FEF3FEF4FEF5FE72AC020E094
:1029900030E040E050E025C02F81388537FDF7CF8B
:1029A0002F31310564F78EE190E0821B930B29856E
:1029B0003A854B855C8504C0569547953795279594
:1029C0008A95D2F78E81882361F050954095309595
:1029D00021953F4F4F4F5F4F04C020E030E040E073
:1029E00050E8CA01B901E2E02C960C944C174F92C2
:1029F0005F926F927F928F929F92AF92BF92DF927F
:102A0000EF92FF920F931F9320E030E040E050E000
:102A1000FC01E480F58006811781D18080818230BD
:102A200038F4D801C701A061AF77B0706FEFD9C09B
:102A3000843009F46EC0823009F471C0E114F104ED
:102A40000105110509F46BC0828193816FEF823813
:102A500096070CF06AC062E87FEF681B790B6A3159
:102A600071050CF080C047015801062E04C0B694D1
:102A7000A794979487940A94D2F74424552432015A
:102A800081E090E0A0E0B0E004C0880F991FAA1F89
:102A9000BB1F6A95D2F70197A109B109E822F92273
:102AA0000A231B23E114F1040105110529F061E05B
:102AB000462E512C612C712C85017401E428F528D7
:102AC00006291729D801C7018F779070A070B070C0
:102AD00080349105A105B10509F457C0D801C7019B
:102AE000CF96A11DB11D60E070E08030E0E09E0750
:102AF000E0E0AE07E0E4BE0710F061E070E027E040
:102B0000B695A795979587952A95D1F7AF77B07029
:102B100068C080E090E0A0E0B0E06FEF62C080E0CD
:102B200090E0A0E0B0E060E05CC0803891058CF7F8
:102B3000BC0161587F4FD801C7018F779070A0709A
:102B4000B07080349105A105B105A1F08FE390E04C
:102B5000A0E0B0E0E80EF91E0A1F1B1F17FD28C0F9
:102B6000D801C701CCCF60E070E080E090E0A0E049
:102B7000B0E0CCCFE7FEF2CF80E490E0A0E0B0E0A0
:102B8000E80EF91E0A1F1B1FE9CFE7FC18C080E002
:102B900090E060E0E61660E0F60660E0060760E4BC
:102BA000160710F081E090E0BC01D801C701A7CF63
:102BB00016950795F794E7946F5F7F4FD1CFD801B3
:102BC000C701805C9F4FAF4FBF4F60E070E0803027
:102BD000E0E09E07E0E0AE07E0E4BE0708F48FCF38
:102BE0008CCF282F392F9A2F9F77842F8078892B8D
:102BF000962F9795992797958F77482F492B66950C
:102C0000852F8078862BD794DD24D7948F77582F03
:102C10005D29CA01B9011F910F91FF90EF90DF90DC
:102C2000BF90AF909F908F907F906F905F904F90EC
:102C30000895FC01DB01208131819281492F4F777A
:102C400050E0991F9927991F8381682F660F692B80
:102C5000881F8827881FFD018183662309F049C0EA
:102C6000211531054105510509F470C082E89FEF37
:102C7000FD0193838283220F331F441F551F220FB0
:102C8000331F441F551F220F331F441F551F220F90
:102C9000331F441F551F220F331F441F551F220F80
:102CA000331F441F551F220F331F441F551F83E03E
:102CB0008C932030F0E03F07F0E04F07F0E45F072F
:102CC00090F482E89FEF220F331F441F551F019796
:102CD000203060E0360760E0460760E4560798F36E
:102CE000FD0193838283FD012483358346835783CB
:102CF00008956F3F71F1862F99278F579040FD01FE
:102D00009383828383E08C93220F331F441F551FCC
:102D1000220F331F441F551F220F331F441F551FFF
:102D2000220F331F441F551F220F331F441F551FEF
:102D3000220F331F441F551F220F331F441F551FDF
:102D400050642483358346835783089582E08C93AF
:102D50000895211531054105510519F484E08C933E
:102D6000089544FD02C01C92BECF81E08C93BBCF7E
:102D7000FB01DC010D900020E9F711974150504014
:102D800028F0019000200D92C9F708951C92089533
:102D9000FB019F01E8944230C4F04532B4F44A305C
:102DA00029F497FB1EF4909581959F4F642F772708
:102DB0000E94F916805D8A330CF0895D8193CB0106
:102DC0000097A1F716F45DE251931082C9010C94AB
:102DD000E916DC01FC0101900020E9F73297AE17FB
:102DE000BF0730F47C916081708331976D93F7CF8A
:102DF0000895AA1BBB1B51E107C0AA1FBB1FA61742
:102E0000B70710F0A61BB70B881F991F5A95A9F793
:102E100080959095BC01CD01089597FB092E07265A
:102E20000AD077FD04D0E5DF06D000201AF47095B3
:102E300061957F4F0895F6F7909581959F4F08957E
:102E40002F923F924F925F926F927F928F929F92BA
:102E5000AF92BF92CF92DF92EF92FF920F931F93A8
:102E6000CF93DF93CDB7DEB7CA1BDB0B0FB6F89459
:102E7000DEBF0FBECDBF09942A88398848885F8499
:102E80006E847D848C849B84AA84B984C884DF800A
:102E9000EE80FD800C811B81AA81B981CE0FD11DEE
:102EA0000FB6F894DEBF0FBECDBFED0108955523D8
:102EB00019F0992351F018C09923A1F097FB6BEDFD
:102EC0007FE089EC9FE397F90895552359F02AF4A0
:102ED0006BED7FE089E490E40895662777278827E3
:102EE000992708950C948A171F93112797FD116055
:102EF00057FD12600E9484130E94D01711FF08C072
:102F00002BED3FE049E450E410FD50680E948E171D
:102F10001F9108959FEF80EC08955058192EC7D047
:102F200001D07AC0BA176207730784079507B1F119
:102F300088F40EF410940B2EBA2FA02D062E622FBB
:102F4000202D072E732F302D082E842F402D092E73
:102F5000952F502DFF275523B9F0591B49F0573EA7
:102F600098F0469537952795A795F0405395C9F762
:102F700076F0BA0F621F731F841F30F48795779520
:102F80006795B795F040939517FA0F2E0895BF1BDC
:102F9000BB27BA0B620B730B840BF6CFDEF6B3C004
:102FA0001F930F930027192F10789F775FE340E856
:102FB000613071058407950718F000680E94FF17BB
:102FC000912B6F937F938F939F930E948518ECE7CB
:102FD000F0E03AD05F914F913F912F910E9466129D
:102FE000002351F02BED3FE049EC5FE300E8902730
:102FF00017FD50680E948E170F911F9108959B0135
:10300000AC019FE380E8772766270C9484139A9598
:10301000BB0F661F771F881F11249923A1F08823F7
:10302000B2F79F3F59F0BB0F48F421F4002011F490
:1030300060FF04C06F5F7F4F8F4F9F4F881F979532
:10304000879597F908955CC0FF92EF92DF92CF9237
:10305000BF926B017C01B59016D0B590BB2069F092
:103060009F938F937F936F93B601C7010CD02F91DD
:103070003F914F915F910E948413BF90CF90DF905A
:10308000EF90FF90089545D002C09601A701EF93FD
:10309000FF930E946612FF91EF913BD0EF93FF9355
:1030A0000E948E17FF91EF91BA9479F70895052E3B
:1030B000092607FA440F551F5F3F79F0AA27A51785
:1030C00008F051E04795880F991F9F3F31F0BB27CB
:1030D000B91708F091E0879508959F919F91112469
:1030E00019CF97FB880F991F9F3F31F0BB27B91766
:1030F00008F091E0879508959F919F9111240ACF40
:10310000662777278827992708959B01AC010C949F
:0C31100066125591459135912591089566
:10311C0055555555555555AAAAAAAAAAAAAAFFFFAC
:10312C00FFFFFFFFFFFFFFFFFFFFFFFF23234062B7
:10313C004570696C657073792056657273696F6E32
:10314C0020302E363023000D0A0154000000000000
:10315C00000A015000000000000A000540000000B9
:10316C00000A000015000000000A000000540000D6
:10317C00000A000000015000000A00000000054099
:10318C00000A000000000015000A017102DA0F4964
:0C319C004096020000000000000000004F
:00000001FF
